:10000000A2EF19F000000000A0EF18F000000000BF
:0C00100000000000000000006AEF19F082
:08001C000AAE029E000E120064
:100024000B840BAE1DEF00F0010E036E026A016A31
:0A003400006A0A360232FF0E1200C5
:10003E000B820BAE29EF00F00368026801680068BE
:08004E000A360232FF0E120017
:0E005600026A016A006A086A036A000E12005C
:100064000CB074EF00F00CA21AEF01F00E6A000E4F
:1000740002648BEF00F0F00E0214D8A456EF00F0E7
:10008400023A01380F0B02260138F00B016E0038DA
:100094000F0B01260038F00B006E08380F0B0026FA
:1000A4000838F00B086E0E84D89002BE6FEF00F093
:1000B40008360036013602360E2A02BE6FEF00F013
:1000C40008360036013602360E2A02BE6FEF00F003
:1000D40008360036013602360E2A0E50036410EF3D
:1000E40001F0035E0BBC08AE15EF01F0D880800E62
:1000F40008640030000E002201220222D8A015EF6D
:1001040001F0023201320032034A1AEF01F015EF16
:1001140001F001C002F000C001F008C000F0086A5C
:10012400000E0E860264C2EF00F0F00E0214D8A492
:10013400AAEF00F0023A01380F0B02260138F00B47
:10014400016E00380F0B01260038F00B006E0E8490
:10015400D89002BE6FEF00F00036013602360E2A48
:1001640002BE6FEF00F00036013602360E2A02BEE0
:100174006FEF00F00036013602360E2A6FEF00F002
:1001840001C002F000C001F0006A000E0E960E8855
:100194000264EFEF00F0F00E0214D8A4DAEF00F0DE
:1001A400023A01380F0B02260138F00B016E0E845F
:1001B400D89002BE6FEF00F0013602360E2A02BE5E
:1001C4006FEF00F0013602360E2A02BE6FEF00F028
:1001D400013602360E2A6FEF00F001C002F0016A08
:1001E400000E0E8602641FEF01F0F00E0214D8A474
:1001F400FEEF00F0023A0E84D89002BE6FEF00F0DA
:1002040002360E2A02BE6FEF00F002360E2A02BE3C
:100214006FEF00F002360E2A6FEF00F0010E0C6E45
:10022400FFDE22EF01F0020E0C6EF6DE22EF01F08B
:10023400040E0C6E02DF22EF01F0080E0C6E09DFD3
:020244001200A6
:080246000B6A0B86FF0E12008B
:10024E000A6A0350D8A40A800750D8A40A820A501A
:10025E00D8B48AEF01F0030AD8B443EF01F00AB024
:10026E003EEF01F006AE88EF01F086EF01F002AE30
:10027E0086EF01F088EF01F00250800B0A6E029EAD
:10028E000650800B069E0A18D8B454EF01F00A509F
:10029E00D8B486EF01F088EF01F00750035CD8B4B4
:1002AE005EEF01F0D8A07AEF01F080EF01F006507A
:1002BE00025CD8B468EF01F0D8A07AEF01F080EFBD
:1002CE0001F00550015CD8B472EF01F0D8A07AEFBE
:1002DE0001F080EF01F00450005CD8B48AEF01F019
:1002EE00D8B080EF01F00A52D8B488EF01F086EF53
:1002FE0001F00A52D8B486EF01F088EF01F0D880F1
:0E030E001200D8901200D880D884120012007D
:10031C000B800BAE9AEF01F0026A0AAEFF0E026E72
:0C032C00016E006E0A360232FF0E120055
:10033800025006180E6E086A096A0B6A03500764B1
:100348008FEF02F006500A6E068E028E03500B6E77
:100358000750036E000E0B64DFEF01F00B50075ED1
:10036800D8B480EF02F0070E07644EEF02F0075E84
:1003780000C008F001C000F002C001F0026A074E98
:1003880080EF02F0076423EF02F0075E00C008F078
:1003980001C000F0016A074E80EF02F0076401EF28
:1003A80002F0075E00C008F0006A074E80EF02F016
:1003B8000764E8EF01F00AC002F005C001F004C0CC
:1003C80000F0086AA9EF03F0030E0764F3EF01F0E9
:1003D800075E08380F0B086E074E80EF02F0D890C2
:1003E8000832074E80EF02F0D8900832074E80EFAF
:1003F80002F0D890083280EF02F0030E076412EF83
:1004080002F0075E08380F0B086E0038F00B08265C
:1004180000380F0B006E074E80EF02F0D8900032C4
:100428000832074E80EF02F0D89000320832074EAB
:1004380080EF02F0D8900032083280EF02F0030E0D
:1004480007643AEF02F0075E08380F0B086E0038B1
:10045800F00B082600380F0B006E0138F00B002651
:1004680001380F0B016E074E80EF02F0D890013271
:1004780000320832074E80EF02F0D8900132003285
:100488000832074E80EF02F0D8900132003208326D
:1004980080EF02F0030E07646BEF02F0075E083886
:1004A8000F0B086E0038F00B082600380F0B006E93
:1004B8000138F00B002601380F0B016E0238F00BE3
:1004C800012602380F0B026E074E80EF02F0D8901B
:1004D8000232013200320832074E80EF02F0D89023
:1004E8000232013200320832074E80EF02F0D89013
:1004F8000232013200320832096A000E0EAE74EF81
:1005080003F0081E001E011E021E082A00220122F6
:10051800022274EF03F00750D8A495EF02F0A9EF78
:1005280003F0096A02C00AF0028E068E0750035CC7
:10053800076ED8B467EF03F0070E076435EF03F0D2
:10054800075E0450096E0550046E0650056E066A73
:10055800074E67EF03F0070E07640AEF03F0075E24
:100568000450096E0550046E056A074E67EF03F0E4
:10057800070E0764E8EF02F0075E0450096E046A8C
:10058800074E67EF03F0070E0764CFEF02F00AC0CB
:1005980002F0A9EF03F0030E0764DAEF02F0075E3A
:1005A80009380F0B096E074E67EF03F0D890093230
:1005B800074E67EF03F0D8900932074E67EF03F054
:1005C800D890093267EF03F0030E0764F9EF02F0E1
:1005D800075E09380F0B096E0438F00B092604383A
:1005E8000F0B046E074E67EF03F0D8900432093200
:1005F800074E67EF03F0D89004320932074E67EFD1
:1006080003F0D8900432093267EF03F0030E076451
:1006180021EF03F0075E09380F0B096E0438F00B61
:10062800092604380F0B046E0538F00B042605382C
:100638000F0B056E074E67EF03F0D89005320432B2
:100648000932074E67EF03F0D890053204320932B9
:10065800074E67EF03F0D89005320432093267EF8E
:1006680003F0030E076452EF03F0075E09380F0B1F
:10067800096E0438F00B092604380F0B046E053890
:10068800F00B042605380F0B056E0638F00B05260F
:1006980006380F0B066E074E67EF03F0D890063248
:1006A800053204320932074E67EF03F0D89006325C
:1006B800053204320932074E67EF03F0D89006324C
:1006C800053204320932086A000E0EAE74EF03F0E8
:1006D800091E041E051E061E092A042205220622DA
:1006E8000950082604500022055001220650022213
:1006F8000EBE8BEF03F0D8A09AEF03F0023201325E
:1007080000320832033E9AEF03F0A4EF03F0D8B0AA
:100718009FEF03F0000E081E001E011E021E082A8D
:100728000022012202220A7E9FEF03F0010E0C6EC6
:1007380095DCABEF03F0020E0C6E90DCABEF03F030
:10074800040E0C6E78DCABEF03F0000E0C6E12009A
:1007580003500718D8A4C0EF03F002500618D8A415
:10076800C0EF03F001500518D8A4C0EF03F0005003
:0E0778000418D8B4D8841200D89412001200CD
:10078600086A096A000E0762036448EF04F0025023
:1007960006180A6E075003267E0ED8A0D9EF03F07E
:1007A600035ED8B04DEF04F0DDEF03F0035ED8A092
:1007B60052EF04F0028E068E02C00EF001C00BF05E
:1007C60000C00DF000500402F4CF0CF001500502F9
:1007D600F4CF00F0F3CF08F00402F3500C26F450E7
:1007E6000822000E00220D500502F3500C26F4508C
:1007F6000822000E002202500402F3500826F4508C
:10080600002202500502016A000E0122F350002662
:10081600F45001220D500602F3500826F45000222F
:10082600026A000E012202220B500602F350002635
:10083600F4500122000E02220E500602F350012649
:10084600F450022202BE30EF04F0083600360136BC
:1008560002360306D8B452EF04F043EF04F0D88012
:10086600800E08640030000E002201220222D8A069
:1008760043EF04F0023201320032034A4DEF04F036
:100886000AAE029E000E55EF04F0010E2BEC00F0AE
:1008960055EF04F0020E1FEC00F055EF04F0040EC5
:0608A60012EC00F012004C
:1008AC00220E0C6E086A096A0A6A0B6A0C06D8B426
:1008BC001FD0D8900B320A3209320832033202327E
:1008CC0001320032D8A0F2D70C06D8B409D00450AB
:1008DC0008260550092206500A2207500B22EAD797
:1008EC00045008260550092206500A2207500B22F4
:0208FC001200E8
:1008FE000601AC51390806E3300EAC5D03E3010E80
:08090E00006E01D0006A120026
:100916000601AC51200A09E0AC510D0804E3090EAA
:10092600AC5D01E302D0006A02D0010E006E120037
:100936000C6A0E6A0250D8A4B4EF04F001C002F0AB
:1009460000C001F0006A0E860250D8A4B4EF04F08D
:1009560001C002F0016A0E960E880250D8B4C6EFA6
:1009660004F00E50035ED8A4D8A0CCEF04F0D890C3
:1009760002BED2EF04F0003601360236032EBBEF7C
:1009860004F0CCEF04F0010E0C6E2BEC00F0D6EF69
:1009960004F0020E0C6E12EC00F0D6EF04F0040E1A
:0809A6000C6E0EEC00F01200D3
:1009AE006DB409D01F0E6B14016E0150000A03E1E5
:0A09BE00010E006E01D0006A120065
:1009C8000050086E0150006E0250016E0350026E16
:1009D800036A0B6A0C6A9E0E036E0A6A02AE01EF86
:1009E80005F0081E001E011E021E082AD8B4002A9F
:1009F800D8B4012AD8B4022A0A8E020E0C6E32EC40
:040A080000F01200E8
:0A0A0C006B826BA201D0FDD712002F
:040A16006B841200DB
:100A1A000601A351A41108E0A3C6E1FFA4C6E2FFA0
:100A2A00A1C6E6FFA2C6E6FFA1C6E9FFA2C6EAFF83
:100A3A00EECF00F000C0A7F600C0ACF667DF0052A8
:100A4A0003E0A14BA22BF0D7A56B000EA7BFFF0EA8
:100A5A00006E000E001802E12D0EA71905E1010E25
:100A6A00A56FA14BA22B0CD0000EA7BFFF0E006EE4
:100A7A00000E001802E12B0EA71902E1A14BA22BCE
:100A8A00A76BA86BA96BAA6BAB6BA66BA5B90BD0AE
:100A9A00A1C6E9FFA2C6EAFFEE502E0A04E1A58923
:100AAA00A14BA22B52D0A1C6E9FFA2C6EAFFEECF04
:100ABA00ACF620DF005201E149D0A583A751080A0C
:100ACA003FE0A5A901D0A607A72BA8C600F0A9C692
:100ADA0001F0AAC602F0ABC603F00A0E046E000EBD
:100AEA00056E066E076EDDDE00C0A8F601C0A9F627
:100AFA0002C0AAF603C0ABF600000000A1C6E9FFD7
:100B0A00A2C6EAFF300EEE5C006E016A000E015AC0
:100B1A00000E01BEFF0E026E036EA8510026A951F7
:100B2A000122AA510222AB51032200C0A8F601C039
:100B3A00A9F602C0AAF603C0ABF60000000003D073
:100B4A00A5B901D0A62BA14BA22BA0D7A76BA1C6F2
:100B5A00E9FFA2C6EAFFEE50650A08E0A1C6E9FF6E
:100B6A00A2C6EAFFEE50450A01E065D0A14BA22BCE
:100B7A00A1C6E9FFA2C6EAFFEE502D0A04E1A58745
:100B8A00A14BA22B09D0A1C6E9FFA2C6EAFFEE50EB
:100B9A002B0A02E1A14BA22BA1C6E9FFA2C6EAFFDA
:100BAA00EE50300A03E1A14BA22BF6D7A1C6E9FF0A
:100BBA00A2C6EAFFEECFACF69DDE005237E0A1C630
:100BCA00E9FFA2C6EAFF300EEE5CA76FA14BA22B8B
:100BDA00A1C6E9FFA2C6EAFFEECFACF68BDE005251
:100BEA0025E00A0EA703F3CFA7F6A1C6E9FFA2C61E
:100BFA00EAFF300EEE5C006E0050A727A14BA22B35
:100C0A00A1C6E9FFA2C6EAFFEECFACF673DE005238
:100C1A000DE00A0EA703F3CFA7F6A1C6E9FFA2C605
:100C2A00EAFF300EEE5C006E0050A727A5A703D09E
:100C3A00A7510008A76FA751A627000EA41902E121
:100C4A00000EA3190AE0A5A308D0A3C6E1FFA4C613
:100C5A00E2FFA1C6E6FFA2C6E6FFA8C600F0A9C643
:100C6A0001F0AAC602F0ABC603F0A9DE00C0A8F6DE
:100C7A0001C0A9F602C0AAF603C0ABF6046A056A67
:100C8A00066A076AA8C600F0A9C601F0AAC602F059
:100C9A00ABC603F05CDD010ED8A4000E006E005254
:100CAA0005E0006A016A026A036A00D1800EA61989
:100CBA00006E800E000A005CD8B071D0A651000800
:100CCA00A66F800EA619006E800E0A0A005C1CE34D
:100CDA00A8C600F0A9C601F0AAC602F0ABC603F086
:100CEA00FF0E046EE60E056E5B0E066E5D0E076E57
:100CFA0045DD00C0A8F601C0A9F602C0AAF603C0E5
:100D0A00ABF60A0EA65FDDD7A651000A1BE0A8C6FD
:100D1A0000F0A9C601F0AAC602F0ABC603F0CD0ED8
:100D2A00046ECC0E056E4C0E066E7B0E076E26DD2B
:100D3A0000C0A8F601C0A9F602C0AAF603C0ABF625
:100D4A00A607E2D7010E046E000E056E000E066EAF
:100D5A00010E076EA8C600F0A9C601F0AAC602F0E5
:100D6A00ABC603F027EC01F0010ED8B0000E006EFE
:100D7A00005214E0A5A109D0010E006E000E016E0A
:100D8A00800E026E030E036E91D0010E006E000EED
:100D9A00016E000E026E010E036E88D070D0800EB6
:100DAA00000A006E800EA619005C69E20A0EA65DB2
:100DBA001CE3A8C600F0A9C601F0AAC602F0ABC699
:100DCA0003F0F90E046E020E056E150E066EA00EE5
:100DDA00076ED4DC00C0A8F601C0A9F602C0AAF6C4
:100DEA0003C0ABF60A0EA65FE1D7A651000A1BE0C4
:100DFA00A8C600F0A9C601F0AAC602F0ABC603F065
:100E0A00000E046E000E056E200E066E820E076E30
:100E1A00B5DC00C0A8F601C0A9F602C0AAF603C054
:100E2A00ABF6A607E2D7A8C604F0A9C605F0AAC67B
:100E3A0006F0ABC607F0FF0E006EFF0E016E7F0EC6
:100E4A00026EFF0E036E27EC01F0010ED8B0000E01
:100E5A00006E005214E0A5A109D0FF0E006EFF0E2D
:100E6A00016EFF0E026EFF0E036E20D0FF0E006EA3
:100E7A00FF0E016E7F0E026EFF0E036E17D0A5A144
:100E8A000DD0000EA819006E000EA919016E800E71
:100E9A00AA19026E000EAB19036E08D0A8C600F09C
:0E0EAA00A9C601F0AAC602F0ABC603F0120002
:100EB8000601A16BA26BA251120802E1A1518E0892
:100EC80008E371DD005201E004D00601A14BA22B1A
:100ED800F2D70601120EA25D02E18F0EA15D03E3B7
:100EE8007B0E006E05D06B806BA001D0FDD7006A29
:020EF8001200E6
:100EFA0000C008F00150006E016A026A036A0B6AB8
:100F0A000C6A016A026A036A960E036E0A6A00AEE6
:100F1A0095EF07F0081E001E082AD8B4002A0A8E88
:100F2A0000C001F008C000F0086A026AFFDC120083
:0E0F3A00ADB202D00000FCD7A1C6AEFF12007F
:100F48000B6A0A6A096A00500402F4CF09F0F3CF69
:100F580008F001500502F4CF0BF0F3CF0AF000506F
:100F68000502F3500926F4500A22E86A0B220150C0
:100F78000402F3500926F4500A22E86A0B2208C03A
:100F880000F009C001F00AC002F00BC003F0120023
:100F9800086A080E0C6E003408360450085ED8B093
:0E0FA80002D00826D89000360C2EF5D7120085
:100FB6000B6A0C6A086A0350D8B45FEF08F002C0E7
:100FC6000AF0028E9E0E035E03AE4FEF08F0036C2E
:100FD600080E035CD8A01CEF08F0036E083600C0AC
:100FE60008F001C000F002C001F0026A080E035CBE
:100FF600D8A01CEF08F0036E083600C008F001C048
:1010060000F0016A080E035CD8A01CEF08F0036E1E
:10101600083600C008F0006A080E035CD8A01CEF72
:1010260008F0036E0836086A0350D8A4D89028EF53
:1010360008F00350D8B428EF08F0D89002320132F5
:1010460000320832032E20EF08F00BBC08A039EF5F
:1010560008F0D8A039EF08F0082AD8B4002AD8B486
:10106600012AD8B4022A02BE63EF08F00AAE5FEF87
:1010760008F0021E011E001E081E082AD8B4002A07
:10108600D8B4012AD8B4022A5FEF08F0026A016ACE
:10109600006A086A5FEF08F00B800BAE6AEF08F093
:1010A600026A0AAE6AEF08F0026E016E006E086E02
:1010B6000A3602326AEF08F00C6A000E6BEF08F08F
:1010C600010E0C6E000E8EEC01F06BEF08F0FF0EB9
:1010D6000250036E0150026E0050016E0850006E01
:0210E6001200F6
:0810E800067E9CEC01F01200F1
:1010F000A49EA1C66FFF6DA401D0FDD7A4BE01D0F0
:10110000FDD76BBC02D0006A03D06B84020E006E68
:021110001200CB
:101112000B6A0350D8B4CFEF08F002500A6E028E69
:101122008E0E035E03AED3EF08F0036C080E035C71
:10113200D8A0AEEF08F0036E013602C001F0026AD9
:10114200080E035CD8A0AEEF08F0036E0136016A08
:101152000350D8A4D890B8EF08F00350D8B4B8EF31
:1011620008F0D89002320132032EB2EF08F00BBC25
:1011720001A0C5EF08F0D8A0C5EF08F0012AD8B445
:10118200022A02BEE2EF08F00AAEE8EF08F0021E01
:10119200011E012AD8B4022AE8EF08F0026A016AA5
:1011A200E8EF08F00B800BAEECEF08F0026A0AAE33
:1011B200ECEF08F0FF0E026E016E0A360232ECEF1F
:1011C20008F0010E0C6E8EEC01F0EEEF08F0000E4E
:1011D2000C6EEEEF08F0FF0E0C6E0150006E025026
:0411E200016E120088
:1011E6000450000A12E10550000A0FE10650000AF9
:1011F6000CE10750000A09E1FF0E006EFF0E016EBA
:101206007F0E026EFF0E036EA8D0086A096A0750A9
:10121600D8B49EEF09F00350D8B4A3EF09F00250FA
:1012260006180A6E028E068E0E6A02C008F001C00B
:101236000CF000C00DF004500D5E0550D8A0053C22
:101246000C5E0650D8A0063C085E086A0C6A0D6A59
:10125600D8A035EF09F0D8900232013200320832B8
:10126600010E0E6E0750035ED8A042EF09F07E0E07
:101276000E240326D8B0A8EF09F048EF09F07E0E39
:101286000E240326D8A0ADEF09F0180E0B6E0D360E
:101296000C3608360036013602360E360450005E2D
:1012A6000550D8A0053C015E0650D8A0063C025E5B
:1012B60006340E120EA063EF09F00D806EEF09F0F2
:1012C600045000260550D8B0053C01260650D8B07B
:1012D600062802260D900B2E4AEF09F094EF09F02E
:1012E600D8900036013602360E360450005E0550A0
:1012F600D8A0053C015E0650D8A0063C025E063426
:101306000E10010B0D26D8B00C2AD8B4082AD8A482
:1013160094EF09F008320C320D32032AD8B4A8EF44
:1013260009F00AAE089E0850026E0C50016E0D5070
:10133600006EB0EF09F0010E23EC01F0B0EF09F0FA
:10134600020E2BEC00F0B0EF09F0040E1FEC00F0DB
:0C135600B0EF09F0080E12EC00F01200DD
:101362008AC6A1F68BC6A2F60601A36BA46B0DEC8E
:0413720005F0120070
:101376008AC604F08BC605F004C0E9FF05C0EAFF83
:10138600EE5203E0044A052AF7D704C002F005C06E
:1013960003F0044A052A8CC600F08DC601F006014A
:1013A6008C4B8D2B00C0E9FF01C0EAFF02C0E1FFB4
:1013B60003C0E2FFEECFE6FF02C0E9FF03C0EAFF8B
:1013C600EE5201E0E2D78AC600F08BC601F01200A9
:1013D6008AC6E9FF8BC6EAFFEECF8CF6000E060141
:1013E6008D6F000E8D6F000E8D1902E1200E8C1987
:1013F60007E0000E8D1902E1090E8C1901E003D0F9
:101406008A4B8B2BE5D78E6B8F6B906B916B000E97
:101416008D1902E12D0E8C1905E1904B912B8A4B0B
:101426008B2B08D0000E8D1902E12B0E8C1902E1D0
:101436008A4B8B2B8AC6E9FF8BC6EAFFEECF8CF66A
:10144600000E8D6F000E8D6F8CC6ACF67FEC04F02F
:10145600005218E08EC600F08FC601F00A0E046E28
:10146600000E056E6EDD300E8C5D026E000E8D591F
:10147600036E025000248E6F035001208F6F8A4B3B
:101486008B2BD8D79051911108E08E510008006E31
:101496008FC601F0000E015604D08EC600F08FC62E
:0414A60001F012003F
:1014AA008DC600F0016A026A036AFF0E0016000E7A
:1014BA00011600C092F601C093F67F0E005C026E20
:1014CA00000E0158036E02C092F603C093F6800E16
:1014DA000318006E800E005C02E1000E025C22E23C
:1014EA00046A056A066A076A8AC600F08BC601F0B2
:1014FA008CC602F08DC603F027EC01F0010ED8B0BD
:10150A00000E006E005209E0000E006E000E016E21
:10151A00800E026E7F0E036E5CD0006A016A026A58
:10152A00036A57D0000E006E06019351005C02E177
:10153A009251180809E28AC600F08BC601F08CC6DF
:10154A0002F08DC603F045D08AC600F08BC601F0C2
:10155A008CC602F08DC603F029DDE4EC04F000C06D
:10156A008EF601C08FF602C090F603C091F600C055
:10157A0004F001C005F002C006F003C007F08AC6F5
:10158A0000F08BC601F08CC602F08DC603F027EC82
:10159A0001F0010ED8B0000E006E005212E0000EEB
:1015AA00046E000E056E000E066E7F0E076E8EC666
:1015BA0000F08FC601F090C602F091C603F08FDDED
:1015CA0008D08EC600F08FC601F090C602F091C610
:0415DA0003F0120008
:1015DE006CDC43C3A1F685DD0601A16B82DD000E36
:1015EE00006E06018D51005C03E18C510301445DD8
:1015FE0005E244C38CF6000E06018D6F0FD0060176
:10160E008C51800FA16FA1076CDD16D006018C5195
:10161E00C00FA16FA10765DD0FD00ED0000E060121
:10162E008B1902E1010E8A19EAE0000E8B1902E114
:10163E00020E8A19EBE0F1D706EC05F043C3A1F6D2
:10164E0050DD400E0601A16F4CDD8CC690F68DC6A6
:10165E0091F68EC6E9FF8FC6EAFFEE521AE08EC6ED
:10166E00D9FF8FC6DAFFDE50800F0601A16F39DD7C
:10167E0006018E4B8F2B904B912B800E006E800EA1
:10168E009119005C03E190510301445D01E201D028
:08169E00E0D70BEC05F012008F
:1016A6008AC604F08BC605F004C002F005C003F03C
:1016B600044A052A8CC600F08DC601F006018C4B43
:1016C6008D2B00C0E9FF01C0EAFF02C0E1FF03C0A5
:1016D600E2FFEECFE6FF02C0E9FF03C0EAFFEE52EB
:0E16E60001E0E2D78AC600F08BC601F01200C8
:1016F40006018D6B8AC6E9FF8BC6EAFFEECF8CF636
:101704008C51000A0EE08CC6A1F615DC06018D2B67
:101714008D518A25E96E000E8B21EA6EEECF8CF690
:04172400EFD71200E9
:101728000D0E0601A16F05DC0A0E0601A16F01DC92
:0217380012009D
:10173A00086A096A100E0C6E01340836093604501C
:10174A00085E0550D8A0053C095ED8B007D0045001
:10175A0008260550D8B0053C0926D890003601362F
:06176A000C2EEAD712006C
:1017700006018D6B030E8D5D0AE28D518B25E16EA6
:10178000000E8C21E26E200EE66E8D2BF3D78D516C
:101790008B25E16E000E8C21E26EE66A8D078D517D
:1017A0008B258E6F000E8C218F6F0A0E046E8AC6F9
:1017B00000F0CCEC07F008C000F0300E00268EC61A
:1017C000E1FF8FC6E2FF00C0E6FF0A0E046E8AC684
:1017D00000F0CCEC07F000C08AF60050000A01E1EE
:0817E00002D08D07DCD71200D6
:1017E8005CEC07F043C3A1F67FDC0601A16B7CDC4F
:1017F800020E0601A16F78DC0BD0800E0601A16FE6
:1018080073DC14D0C00E0601A16F6EDC0FD00ED0B1
:10181800000E06018B1902E1010E8A19EEE0000E96
:101828008B1902E1020E8A19EDE0F1D706EC05F0FA
:1018380043C3A1F659DC400E0601A16F55DC060131
:101848008C6B8D6B800E8D19006E800E005C04E130
:101858000301445106018C5D07E2A00EA16F44DC30
:1018680006018C4B8D2BEED706EC05F043C3A1F691
:101878003BDC0601A16B38DC0BD0800E0601A16FA2
:1018880033DC14D0C00E0601A16F2EDC0FD00ED0B1
:10189800000E06018B1902E1010E8A19EEE0000E16
:1018A8008B1902E1020E8A19EDE0F1D70BEC05F075
:0218B80012001C
:1018BA0006019051000805E3070E916F000E926F22
:1018CA0012D09051160805E2170E936F000E946F0E
:1018DA0006D09051010F936F946B000E942393C618
:1018EA0091F694C692F691C69BF692C69CF6956BB3
:1018FA00966B046A056A066A076A8AC600F08BC68E
:10190A0001F08CC602F08DC603F027EC01F0010E3F
:10191A00D8B0000E006E005209E08EC6E1FF8FC6F5
:10192A00E2FF2D0EE66E8E4B8F2B8C7F8AC604F05B
:10193A008BC605F08CC606F08DC607F0006A016AF0
:10194A00026A036A27EC01F0010ED8B0000E006E9D
:10195A00005237E0000E046E000E056E000E066E91
:10196A007F0E076E8AC600F08BC601F08CC602F0A5
:10197A008DC603F027EC01F0010ED8B0000E006E00
:10198A0000521FE08AC600F08BC601F08CC602F036
:10199A008DC603F0000E046E000E056E200E066E54
:1019AA00820E076EC3EC03F000C08AF601C08BF604
:1019BA0002C08CF603C08DF6010E955F000E965B91
:1019CA00C9D7000E046E000E056E200E066E820E3A
:1019DA00076E8AC600F08BC601F08CC602F08DC66F
:1019EA0003F027EC01F0000ED8B0010E006E005291
:1019FA001EE0000E046E000E056E200E066E820EAC
:101A0A00076E8AC600F08BC601F08CC602F08DC63E
:101A1A0003F0F3EC08F000C08AF601C08BF602C0AE
:101A2A008CF603C08DF60601954B962BCAD79551B5
:101A3A009B2796519C23010E976F000E986F000EFC
:101A4A009D6F000E9E6F000E9F6F7F0EA06F800E1F
:101A5A009819006E800E9C19005C02E19B51975DFB
:101A6A001EE2000E046E000E056E200E066E820E39
:101A7A00076E9DC600F09EC601F09FC602F0A0C682
:101A8A0003F0F3EC08F000C09DF601C09EF602C018
:101A9A009FF603C0A0F60601974B982BD8D7000EE5
:101AAA00046E000E056E000E066E800E076E9DC651
:101ABA0000F09EC601F09FC602F0A0C603F0F3EC48
:101ACA0008F08AC604F08BC605F08CC606F08DC6EF
:101ADA0007F09CEC01F000C08AF601C08BF602C048
:101AEA008CF603C08DF6000E046E000E056E200EF5
:101AFA00066E820E076E27EC01F0000ED8B0010EBA
:101B0A00006E00520BE0000E06018A6F000E8B6F0A
:101B1A00000E8C6F7F0E8D6F954B962B0601800EF3
:101B2A009619006E800E005C02E1000E955D38E2A7
:101B3A008EC6E1FF8FC6E2FF300EE66E8E4B8F2B0C
:101B4A008EC6E1FF8FC6E2FF2E0EE66E8E4B8F2BFE
:101B5A00800E9C19006E800E005C02E1000E9B5DF7
:101B6A0004E29B51955F9C51965BFF0E976FFF0EA7
:101B7A00986F800E9619006E800E9819005C02E12B
:101B8A009751955D0DE28EC6E1FF8FC6E2FF300EDA
:101B9A00E66E8E4B8F2B010E975F000E985BE9D78E
:101BAA00976B986B800E9819006E800E9C19005CDA
:101BBA0002E19B51975D63E28AC600F08BC601F091
:101BCA008CC602F08DC603F089EC08F000C099F6C5
:101BDA0001C09AF6300E00268EC6E1FF8FC6E2FFDC
:101BEA0000C0E6FF8E4B8F2B9851961902E1955152
:101BFA00971908E18EC6E1FF8FC6E2FF2E0EE66E48
:101C0A008E4B8F2B99C600F09AC601F07DEC07F037
:101C1A0000C09DF601C09EF602C09FF603C0A0F662
:101C2A0000C004F001C005F002C006F003C007F0CE
:101C3A008AC600F08BC601F08CC602F08DC603F08E
:101C4A0074EC08F000C08AF601C08BF602C08CF66C
:101C5A0003C08DF6000E046E000E056E200E066E91
:101C6A00820E076EC3EC03F000C08AF601C08BF641
:101C7A0002C08CF603C08DF6974B982B93D78EC66D
:0A1C8A00E1FF8FC6E2FFE66A1200D8
:101C94008CC604F08DC605F08AC602F08BC603F02C
:101CA4008EC600F08FC601F0010E06018E5F000E95
:101CB4008F5B005001100FE004C0E9FF05C0EAFF8C
:101CC40002C0E1FF03C0E2FFEECFE6FF024A032AAF
:101CD400044A052AE5D78AC600F08BC601F0120033
:0E1CE400A8B202D00000FCD78AC6A9FF1200E9
:101CF2008AC602F08BC603F002C000F003C001F0F6
:101D0200024A032A00C0E9FF01C0EAFFEE5201E0E5
:101D1200F3D706018A51025C006E8B510358016EA3
:0A1D2200010E005E000E015A1200CF
:101D2C008AC6F6FF8BC6F7FF8CC6F8FF0900F5CF05
:101D3C0000F0005212E08AC6F6FF8BC6F7FF8CC685
:101D4C00F8FF0900F5CFA1F69DEC07F0010E060196
:0C1D5C008A27000E8B238C23E3D7120093
:101D68008CC6F6FF8DC6F7FF8EC6F8FF0900F5CFC3
:101D780000F0005218E08CC6F6FF8DC6F7FF8EC63D
:101D8800F8FF0900F5CF00F08AC6E1FF8BC6E2FF35
:101D980000C0E6FF06018A4B8B2B010E8C27000E34
:101DA8008D238E23DDD78AC6E1FF8BC6E2FFE66A64
:021DB800120017
:0E1DBA00570E0D6E0D2EFED700000000120019
:101DC8001D0E06018A6F000E8B6F860E8C6F3F0EFC
:101DD8008D6F000E8E6FC4DF72C01DF073C01EF0D1
:101DE80074C020F075C021F076C023F077C024F0CD
:101DF800256A180E06018A6F3F0E8B6F000E8C6FD6
:101E080091DF1D0E06018A6F000E8B6F6FDC090EC5
:101E1800A16F9DEC07F0300E0001725D006E016A43
:101E2800000E015A0A0E046E000E056EA4EC07F0AF
:101E380073510026000E0122300E005C0601726FFD
:101E4800000E0158736F72C639F073C63AF0300E3F
:101E58000001745D006E016A000E015A0A0E046EDC
:101E6800000E056EA4EC07F075510026000E012245
:101E7800300E005C0601706F000E0158716F70C65D
:101E88003BF071C63CF0300E0001765D006E016AD1
:101E9800000E015A0A0E046E000E056EA4EC07F03F
:101EA80077510026000E0122300E005E000E015A06
:101EB80000C0BDF001C0BEF0000E026E036EA00EA1
:101EC800046E860E056E010E066E000E076E56EC49
:101ED80004F000C06CF601C06DF602C06EF603C0D7
:101EE8006FF670C600F071C601F0000E026E036E48
:101EF800640E046E000E056E066E076E56EC04F056
:101F0800005006016C25266E01506D21276E025087
:101F18006E21286E03506F21296E72C600F073C6B9
:101F280001F0000E026E036E005026260150272293
:0E1F3800025028220350292294EC0BF01200D4
:101F4600D10E06018A6F3E0E8B6F000E8C6FEBDE94
:101F56006CC68AF66E0E06018B6F060E8C6F05DC5C
:101F66006E0E8A6F060E8B6F7AEC0BF08F0E8A6FF1
:101F76003F0E8B6F000E8C6FD6DE7D0E06018A6FCC
:101F86003F0E8B6F000E8C6FCEDE5CEC07F06CC6DE
:101F9600A1F678EC08F000C06DF60050000A0BE0E0
:101FA600E10E06018A6F3E0E8B6F000E8C6FBBDE54
:101FB60006016D6B0BD00601730E8A6F3F0E8B6F99
:101FC600000E8C6FB0DE010E06016D6F0BEC05F096
:0A1FD60094EC0BF06DC600F0120051
:101FE00070C600F006017007005228E06CC6E9FFD9
:101FF0006DC6EAFFEE50000A0CE06CC6E9FF6DC644
:10200000EAFF6EC6D9FF6FC6DAFFEE50DE1801E1B7
:102010000FD06CC6E9FF6DC6EAFF6EC6D9FF6FC66A
:10202000DAFFDE50EE5C006E016A000E015A08D045
:1020300006016C4B6D2B6E4B6F2BD2D7006A016A79
:0220400012008C
:102042006CC604F06DC605F006017051711124E0F2
:10205200010E705F000E715B04C002F005C003F058
:10206200044A052A6EC600F06FC601F06E4B6F2B54
:1020720000C0E9FF01C0EAFF02C0E1FF03C0E2FFC6
:10208200EECFE6FF02C0E9FF03C0EAFFEECF00F0A9
:10209200005201E101D0D8D770C600F071C601F03C
:1020A200010E705F000E715B0050011008E004C069
:1020B200E1FF05C0E2FFE66A044A052AEDD76CC6D5
:0820C20000F06DC601F01200F0
:1020CA0006016F6B6CC6E9FF6DC6EAFFEECF6EF6CE
:1020DA006E51000A0EE06EC68AF6FFDD06016F2B0E
:1020EA006F516C25E96E000E6D21EA6EEECF6EF629
:0420FA00EFD712000A
:1020FE003A0E05015F6F0F0E606FA10E616F060E37
:10210E00626FFF0E636FFF0E646F000E656F000E41
:10211E00666FFF0E576FFF0E586F000E596F000E51
:10212E005A6FFF0E5B6FFF0E5C6F000E5D6F000E41
:10213E005E6FAD8A900EAC6E948E949C9EAA03D068
:08214E00AFCF00F0FBD7120037
:10215600FD0EC16EFF0EC26EFF0E926EFF0E936EE7
:10216600FF0E956EFF0E946EFF0E986E959C9284F0
:10217600958E9986959896988C988D98938212004C
:102186000900F5CFE6FF0006FBE10106F9E11200C2
:10219600150E7B6EA00E7A6E0201C16BC26B799230
:1021A600798A7988799C79967994798E7990A292B0
:0621B600A192A0921200AC
:1021BC00959A959C8C9A8C9C958A958C6D9E6D9C11
:0621CC00380E6C6E1200DB
:1021D200E40E05015F6F1C0E606F8A0E616F060EC2
:1021E200626FFF0E636FFF0E646F000E656F000E6D
:1021F200666FFF0E576FFF0E586F000E596F000E7D
:102202005A6FFF0E5B6FFF0E5C6F000E5D6F000E6C
:102212005E6FA88A900E9C6E98849892A4AA03D0AE
:08222200AACF00F0FBD7120067
:10222A0006016E6B6F6B010E726F000E736FC30E39
:10223A008A6F020E8B6F58DD00C070F601C071F60E
:10224A00070E6C6F000E6D6F800E6D19006E800E9A
:10225A007119005C02E170516C5DD8B089D146D128
:10226A00C30E6C25E96E020E6D21EA6EEE502C0A41
:10227A000EE1280E6E25E16E060E6F21E26EE66A09
:10228A006E6B6F6B020E726F000E736F6ED1280E3B
:10229A006E25E16E060E6F21E26EC30E6C25E96EA5
:1022AA00020E6D21EA6EEECFE6FF6E4B6F2B5DD10B
:1022BA00C30E6C25E96E020E6D21EA6EEE502C0AF1
:1022CA000EE14C0E6E25E16E060E6F21E26EE66A95
:1022DA006E6B6F6B030E726F000E736F46D14C0EEE
:1022EA006E25E16E060E6F21E26EC30E6C25E96E55
:1022FA00020E6D21EA6EEECFE6FF6E4B6F2B35D1E3
:10230A00C30E6C25E96E020E6D21EA6EEE502C0AA0
:10231A0007E16E6B6F6B040E726F000E736F25D13F
:10232A00C30E6C25E96E020E6D21EA6EEECF23F61E
:10233A006E4B6F2B1AD1C30E6C25E96E020E6D21FE
:10234A00EA6EEE502C0A0EE1380E6E25E16E060E8C
:10235A006F21E26EE66A6E6B6F6B050E726F000E8E
:10236A00736F03D1380E6E25E16E060E6F21E26E91
:10237A00C30E6C25E96E020E6D21EA6EEECFE6FF02
:10238A006E4B6F2BF2D0C30E6C25E96E020E6D21D7
:10239A00EA6EEE502C0A07E16E6B6F6B060E726FD7
:1023AA00000E736FE2D0C30E6C25E96E020E6D212A
:1023BA00EA6EEECF6BF66E4B6F2BD7D0C30E6C2541
:1023CA00E96E020E6D21EA6EEE502C0A07E16E6B81
:1023DA006F6B070E726F000E736FC7D0C30E6C253A
:1023EA00E96E020E6D21EA6EEECF4DF36E4B6F2B46
:1023FA00BCD0C30E6C25E96E020E6D21EA6EEE505A
:10240A002C0A0EE1190E6E25E16E060E6F21E26EA0
:10241A00E66A6E6B6F6B080E726F000E736FA5D053
:10242A00190E6E25E16E060E6F21E26EC30E6C2543
:10243A00E96E020E6D21EA6EEECFE6FF6E4B6F2B50
:10244A0094D0C30E6C25E96E020E6D21EA6EEE5031
:10245A002C0A0EE1450E6E25E16E030E6F21E26E27
:10246A00E66A6E6B6F6B090E726F000E736F7DD02A
:10247A00450E6E25E16E030E6F21E26EC30E6C25CA
:10248A00E96E020E6D21EA6EEECFE6FF6E4B6F2B00
:10249A006CD0C30E6C25E96E020E6D21EA6EEE5009
:1024AA002C0A0EE1570E6E25E16E060E6F21E26EC2
:1024BA00E66A6E6B6F6B0A0E726F000E736F55D001
:1024CA00570E6E25E16E060E6F21E26EC30E6C2565
:1024DA00E96E020E6D21EA6EEECFE6FF6E4B6F2BB0
:1024EA0044D070C66CF671C66DF63FD0000E7319F3
:1024FA0002E1010E7219D8B4B3D6000E731902E1C3
:10250A00020E7219D8B4D4D6000E731902E1030E62
:10251A007219D8B4F5D6000E731902E1040E7219B5
:10252A00D8B409D7000E731902E1050E7219D8B48E
:10253A002AD7000E731902E1060E7219D8B43ED7D3
:10254A00000E731902E1070E7219D8B452D7000EA1
:10255A00731902E1080E7219D8B473D7000E7319F1
:10256A0002E1090E721995E0BCD76C4B6D2B6CD643
:0A257A0072C600F073C601F01200F3
:102584000001BF6BC06B020EC05D02E1000EBF5DB7
:102594000AE2C10EBF25E16E000EC021E26EE66ABA
:1025A400BF4BC02BF0D705016B6B6C6B0001BF6B8D
:1025B400C06B9EAA02D0AFCF6DF505016D6B696B40
:0625C4006A6BA08A120000
:1025CA00C29EC29CC29AC298C296C284C280FF0EA0
:1025DA00C16EC192C18EC19CC18AC188C196C18295
:0625EA00C194C190120033
:1025F000730E06018A6F060E8B6F70C68CF671C65D
:102600008DF672C68EF6B4EC0EF05CEC07F043C3A8
:10261000A1F678EC08F00601A16B78EC08F0000E4A
:10262000006E06016F51005C03E16E510301445DD1
:1026300005E244C36EF6000E06016F6F11D006016D
:102640006E51800FA16FA10778EC08F017D006013A
:102650006E51C00FA16FA10778EC08F00FD00ED01B
:10266000000E06016D1902E1010E6C19E8E0000E82
:102670006D1902E1020E6C19EAE0F1D706EC05F0E3
:1026800043C3A1F678EC08F0400E0601A16F78EC88
:1026900008F06EC688F66FC689F670C6F6FF71C67A
:1026A000F7FF72C6F8FF0900F5CF00F0005223E0F3
:1026B00070C6F6FF71C6F7FF72C6F8FF0900F5CFC6
:1026C00000F00050800F0601A16F78EC08F0010EB9
:1026D00006017027000E71237223884B892B800E10
:1026E000006E800E8919005C03E188510301445D8E
:0C26F00001E201D0D2D70BEC05F0120083
:1026FC00150E7B6EA00E7A6E0201C16BC26BA1929D
:06270C00A082798012009A
:10271200A70E06018A6F3F0E8B6F000E8C6F96EC30
:102722000EF028C6A1F69DEC07F029C6A1F69DEC95
:1027320007F0480E0601A16F9DEC07F02AC6A1F62C
:102742009DEC07F02BC6A1F69DEC07F04D0E06019D
:10275200A16F9DEC07F02CC6A1F69DEC07F02DC6EB
:10276200A1F69DEC07F0530E0601A16F9DEC07F058
:10277200530E06018A6F3F0E8B6F000E8C6F96EC24
:102782000EF0380E06018A6F060E8B6FB1EC09F05F
:1027920000C034F601C035F602C036F603C037F683
:1027A200000E046E000E056E480E066E850E076E54
:1027B200F3EC08F000C024F601C025F602C026F6AC
:1027C20003C027F600C08AF601C08BF602C08CF661
:1027D20003C08DF655EC0AF000C06CF601C06DF630
:1027E20002C06EF603C06FF66CC624F66DC625F6FF
:1027F2006EC626F66FC627F6000E046E000E056E34
:10280200480E066E850E076E34C600F035C601F01E
:1028120036C602F037C603F0F3EC08F06CC604F0DB
:102822006DC605F06EC606F06FC607F074EC08F0D0
:1028320000C01DF601C01EF602C01FF603C020F63E
:10284200000E046E000E056E480E066E850E076EB3
:10285200C3EC03F0000E046E000E056E700E066EE1
:10286200840E076EF3EC08F06CC604F06DC605F03A
:102872006EC606F06FC607F09CEC01F000C034F69D
:1028820001C035F602C036F603C037F600C08AF63C
:1028920001C08BF602C08CF603C08DF621C68EF6FF
:1028A20022C68FF6060E0601906F5DEC0CF021C673
:1028B2008AF622C68BF67AEC0BF0200EA16F9DEC05
:1028C20007F023C6A1F69DEC07F0300E06018A6FD1
:1028D2003F0E8B6F000E8C6F96EC0EF04C0E0601C5
:1028E2008A6F060E8B6FB1EC09F000C048F601C08A
:1028F20049F602C04AF603C04BF6000E046E000E03
:10290200056E480E066E850E076EF3EC08F000C0E9
:1029120024F601C025F602C026F603C027F600C041
:102922008AF601C08BF602C08CF603C08DF655EC18
:102932000AF000C06CF601C06DF602C06EF603C06C
:102942006FF66CC624F66DC625F66EC626F66FC601
:1029520027F6000E046E000E056E480E066E850EFA
:10296200076E48C600F049C601F04AC602F04BC6DF
:1029720003F0F3EC08F06CC604F06DC605F06EC609
:1029820006F06FC607F074EC08F000C01DF601C037
:102992001EF602C01FF603C020F6000E046E000EE3
:1029A200056E480E066E850E076EC3EC03F0000E30
:1029B200046E000E056E700E066E840E076EF3EC4A
:1029C20008F06CC604F06DC605F06EC606F06FC660
:1029D20007F09CEC01F000C048F601C049F602C0C5
:1029E2004AF603C04BF600C08AF601C08BF602C05D
:1029F2008CF603C08DF621C68EF622C68FF6060E21
:102A02000601906F5DEC0CF021C68AF622C68BF6A9
:102A12007AEC0BF0200EA16F9DEC07F06BC6A1F6CD
:102A22009DEC07F03C0E06018A6F3F0E8B6F000E85
:102A32008C6F96EC0EF0570E06018A6F060E8B6FA6
:102A4200B1EC09F000C067F601C068F602C069F691
:102A520003C06AF600C08AF601C08BF602C08CF68B
:102A620003C08DF621C68EF622C68FF6010E906F38
:102A72005DEC0CF021C68AF622C68BF67AEC0BF0DE
:102A8200480E8A6F3F0E8B6F000E8C6F96EC0EF025
:102A9200190E06018A6F060E8B6F7AEC0BF0240E6C
:102AA2008A6F3F0E8B6F000E8C6F96EC0EF0450E08
:102AB20006018A6F030E8B6F7AEC0BF0690E8A6F38
:102AC2003F0E8B6F000E8C6F96EC0EF04DC3A1F68D
:0A2AD2009DEC07F094EC0BF01200ED
:102ADC0003014E6B4F6B020E4F5D02E1000E4E5D1B
:102AEC000AE2530E4E25E16E030E4F21E26EE66AAA
:102AFC004E4B4F2BF0D70501536B546B03014E6BB0
:102B0C004F6BA4AA02D0AACF50F3506B516B526BEF
:042B1C00A38A120076
:102B200006016E6B6F6B1F0E0B6E710E0C6E1E0E20
:102B30000D6E0D2EFED70C2EFCD70B2EFAD70000F3
:102B40005CEC07F043C3A1F678EC08F000C06CF62B
:102B5000000E06016D6F000E6D1902E1000E6C197A
:102B600005E06EC600F06FC601F0E0D06E4B6F2B33
:102B70000D0E0B6E2D0E0C6ED70E0D6E0D2EFED79C
:102B80000C2EFCD70B2EFAD700000000A16B78ECBE
:102B900008F000C06CF6000E06016D6F800E006E2E
:102BA000800E6D19005C02E16C51000805E26EC6F2
:102BB00000F06FC601F0BAD06E4B6F2B240EA16FE0
:102BC00078EC08F00C0E0601A16F78EC08F0060E08
:102BD0000601A16F78EC08F0250E0601A16F78ECD4
:102BE00008F0060E0601A16F78EC08F0110E060140
:102BF000A16F78EC08F0420E0601A16F78EC08F0A6
:102C0000960E0601A16F78EC08F0240E0601A16F64
:102C100078EC08F000C06CF6000E06016D6F800EB7
:102C2000006E800E6D19005C02E16C51000805E237
:102C30006EC600F06FC601F079D06E4B6F2B0C0E94
:102C4000A16F78EC08F000C06CF6000E06016D6F05
:102C5000800E006E800E6D19005C02E16C51000860
:102C600005E26EC600F06FC601F060D06E4B6F2BB0
:102C7000060EA16F78EC08F000C06CF6000E06019D
:102C80006D6F800E006E800E6D19005C02E16C515C
:102C9000000805E26EC600F06FC601F047D06E4B2B
:102CA0006F2B020EA16F78EC08F000C06CF6000EDE
:102CB00006016D6F800E006E800E6D19005C02E1E2
:102CC0006C51000805E26EC600F06FC601F02ED010
:102CD0006E4B6F2B010EA16F78EC08F000C06CF604
:102CE000000E06016D6F800E006E800E6D19005C87
:102CF00002E16C51000805E26EC600F06FC601F0FB
:102D000015D0070E0B6E170E0C6E6A0E0D6E0D2E83
:102D1000FED70C2EFCD70B2EFAD700000BEC05F0DB
:0E2D20006E4B6F2B6EC600F06FC601F01200F6
:102D2E000601706B050E705D0AE270516E25E16E44
:102D3E00000E6F21E26E200EE66E702BF3D77051EF
:102D4E006E25E16E000E6F21E26EE66A700770511D
:102D5E006E25716F000E6F21726F0A0E046E000EDB
:102D6E00056E6CC600F06DC601F09DEC0BF008C050
:102D7E0000F009C001F0300E002671C6E1FF72C6E8
:102D8E00E2FF00C0E6FF0A0E046E000E056E6CC672
:102D9E0000F06DC601F09DEC0BF000C06CF601C0AA
:102DAE006DF6000E011802E1000E001801E102D0CE
:062DBE007007CDD71200E2
:102DC400020E06018A6F000E8B6FF4EC0BF0010EFD
:0E2DD40006018A6F000E8B6FF4EC0BF01200FC
:102DE200010E06018A6F000E8B6FF4EC0BF0F00EF1
:102DF20006018A6F050E8B6FAF0E8C6F3E0E8D6FC4
:102E0200000E8E6FB4EC0EF0570E06018A6F060E9E
:102E12008B6F79EC0EF000500608026E01C003F0D1
:102E2200000E035602C06CF603C06DF6800E031846
:102E3200006E800E005C02E1000E025C02E26C6B2E
:102E42006D6B6C51FB088A6F6DC68BF6050E8B5746
:102E5200570E8C6F060E8D6F53EC0BF06D0E050145
:102E6200FF6F010E06018A6F000E8B6F010E8C6FD1
:102E7200000E8D6FF00E8E6F050E8F6FEFEC0AF065
:102E8200020E06018A6F000E8B6FF4EC0BF0F00E4F
:102E920006018A6F050E8B6F5A0E8C6F3E0E8D6F78
:102EA200000E8E6FB4EC0EF06E0E06018A6F060EE7
:102EB2008B6F280E8C6F060E8D6F020E8E6F000EBA
:102EC2008F6F4AEC0EF06E0E8A6F060E8B6FEBEC74
:102ED20009F0010E0024026E000E0120036E02C0F2
:102EE20071F603C072F6800E006E800E0318005C4D
:102EF20002E10250170802E2716B726B016A80B440
:102F0200012A0150000A010ED8A4000E006E0050E2
:102F12007127000E7223280E8A6F060E8B6F79ECD2
:102F22000EF000C06CF601C06DF671C68AF66E0E28
:102F32008B6F060E8C6FB8EC0BF0F50E8A6F050ED8
:102F42008B6F6F0E8C6F060E8D6F020E8E6F000EE2
:102F52008F6F4AEC0EF0F80E8A6F050E8B6F2A0EF9
:102F62008C6F060E8D6F020E8E6F000E8F6F4AEC05
:102F72000EF0FB0E8A6F050E8B6F2C0E8C6F060EF9
:102F82008D6F020E8E6F000E8F6F4AEC0EF0006B8B
:102F9200020E8A6F000E8B6F010E8C6F000E8D6F0A
:102FA200F00E8E6F050E8F6FEFEC0AF05C0E0B6E5B
:102FB200510E0C6E600E0D6E0D2EFED70C2EFCD730
:102FC2000B2EFAD70000F00E06018A6F050E8B6FEA
:102FD2006B0E8C6F3E0E8D6F000E8E6FB4EC0EF08A
:102FE20034C68AF635C68BF636C68CF637C68DF6EB
:102FF200F50E06018E6F050E8F6F060E906F5DEC5B
:103002000CF0F00E8A6F050E8B6F79EC0EF0800ECD
:103012000118026E800E025C02E1100E005C0BE2EF
:10302200F00E8A6F050E8B6F2F0E8C6F000E8D6F58
:10303200BBEC09F0E6D76BC6FFF5006B010E8A6F99
:10304200000E8B6F010E8C6F000E8D6FF00E8E6F67
:10305200050E8F6FEFEC0AF0F00E06018A6F050E77
:103062008B6F7C0E8C6F3E0E8D6F000E8E6FB4ECEC
:103072000EF048C68AF649C68BF64AC68CF64BC68F
:103082008DF6F50E06018E6F050E8F6F060E906F90
:103092005DEC0CF0F00E8A6F050E8B6F79EC0EF082
:1030A200800E0118026E800E025C02E1100E005CBE
:1030B2000BE2F00E8A6F050E8B6F330E8C6F000ED3
:1030C2008D6FBBEC09F0E6D723C6FFF5006B020E4D
:1030D2008A6F000E8B6F010E8C6F000E8D6FF00EDB
:1030E2008E6F050E8F6FEFEC0AF05C0E0B6E510EB9
:1030F2000C6E600E0D6E0D2EFED70C2EFCD70B2E15
:06310200FAD700001200E4
:10310800C26A070EC16EC18E6CC600F00036009010
:10311800003600900050C212C280DDEC0EF0C28270
:10312800C2A201D0FDD7C4CF01F0006AC35000127B
:08313800000E0112C29012000A
:1031400000C01AF0E1CF1BF0E2CF1CF09EAA4BD0DA
:103150009DAA49D0ACA203D0AC98AC88AC92ACA4E8
:1031600002D0AFCF6DF5AFCF6DF505016D510D0AF2
:1031700008E0020E0001C05D02E1000EBF5D01E249
:1031800023D0010E0501696F000E6A6F020E000167
:10319000C05D02E1000EBF5D05E3020E0501696F2F
:1031A000000E6A6FA09AC10E0001BF25E16E000EED
:1031B000C021E26EE66ABFC06BF5C0C06CF5BF6BA4
:1031C000C06B05016D6B0FD0C10E0001BF25E16E14
:1031D000000EC021E26E6DC5E6FFBFC06BF5C0C03A
:1031E0006CF5BF4BC02BA4AA6ED0A3AA6CD09CA236
:1031F00002D09C989C889CA402D0AACF50F3AACF5E
:1032000050F3010E03014F5D02E1FF0E4E5D04E23B
:1032100050510D0A01E035D04EC353F54FC354F55C
:10322000A4BA01D0FDD7AACF50F3506B000E5219AB
:1032300002E1000E511908E13D0E4E25E16E000E2F
:103240004F21E26E50C3E6FF000E521902E1010E5B
:10325000511908E1C30E4E25E16E020E4F21E26EB8
:1032600050C3E6FF4E6B4F6B514B522B000E521961
:1032700002E1020E511904E1AACF50F3506BA39A58
:1032800022D0000E521902E1000E511908E13D0E44
:103290004E25E16E000E4F21E26E50C3E6FF000E98
:1032A000521902E1010E511908E1C30E4E25E16EDB
:1032B000020E4F21E26E50C3E6FF4EC353F54FC3DB
:1032C00054F54E4B4F2B1AC000F01BC0E1FF1CC041
:0432D000E2FF110008
:1032D40000C019F001C018F0156ED8CF16F0E0CF79
:1032E40017F0A0A222D0A1A220D0010E355C006E5E
:1032F400000E3658016E00C035F001C036F0150ED0
:103304007B6EA00E7A6E800E006E800E3618005C06
:1033140002E13550000807E3010E0201C16F000EFF
:10332400C26F7990A092A192A1921750E06E1650AC
:10333400D86E153A153819C000F018C001F0100005
:10334400D7EC1FF0D38CD38AD388D382D3909B6AD3
:103354009B8CD3B601D0FDD7ABEC10F0640E356E68
:10336400000E366E6E0E0601216F050E226F0501EA
:103374006E6BF06B020E0A6E310E0B6E620E0C6EEB
:10338400450E0D6E0D2EFED70C2EFCD70B2EFAD744
:103394000A2EF8D77E86010E7F6E370EB06EAD848E
:1033A4007FEC10F00C0E0601A16F9DEC07F01F0ED0
:1033B4000B6E710E0C6E1E0E0D6E0D2EFED70C2EA6
:1033C400FCD70B2EFAD70000A70E06018A6F3B0E1E
:1033D4008B6F000E8C6F96EC0EF0E70E06018A6F71
:1033E4003B0E8B6F000E8C6F96EC0EF0D80E060120
:1033F4008A6F3A0E8B6F000E8C6F96EC0EF0810E76
:1034040006018A6F3C0E8B6F000E8C6F96EC0EF0EB
:103414000A0E06018A6F3E0E8B6F000E8C6F96ECBF
:103424000EF08A0E06018A6F3A0E8B6F000E8C6FB7
:1034340096EC0EF0ED0E06018A6F3C0E8B6F000EBB
:103444008C6F96EC0EF0650E06018A6F3B0E8B6F47
:10345400000E8C6F96EC0EF0870E06018A6F3D0EFF
:103464008B6F000E8C6F96EC0EF00D0E0B6E2D0E06
:103474000C6ED70E0D6E0D2EFED70C2EFCD70B2E18
:10348400FAD7000000007C86020E7D6E700EAB6ED3
:10349400A884E9EC10F01E0E6E6EDEEC10F04E0EF9
:1034A40006018A6F3D0E8B6F000E8C6F96EC0EF04A
:1034B400640E356E000E366ECBEC10F0740E030104
:1034C400436F740E0601186F100E0301446FA70EAC
:1034D40006018A6F3C0E8B6F000E8C6F96EC0EF01B
:1034E40018C66CF6A3EC0FF000C0EEF5000E050153
:1034F400EF6F94EC0BF0220E06018A6F3E0E8B6F79
:10350400000E8C6F96EC0EF090EC15F000C0EEF50A
:1035140001C0EFF50A0E0B6E220E0C6EA10E0D6E9D
:103524000D2EFED70C2EFCD70B2EFAD749DC0A0E33
:103534000B6E220E0C6EA10E0D6E0D2EFED70C2EF0
:10354400FCD70B2EFAD7010E06016C6F000E6D6FBF
:10355400010E6E6F000E6F6FC00E706F3E0E716FB6
:10356400000E726FF8EC12F0020E06016C6F000E82
:103574006D6F010E6E6F000E6F6F380E706F3E0E22
:10358400716F000E726FF8EC12F07A0E0B6EC10EB2
:103594000C6E810E0D6E0D2EFED70C2EFCD70B2E4D
:1035A400FAD700000000640E356E000E366E1F0E52
:1035B40006018A6F3C0E8B6F000E8C6F96EC0EF03A
:1035C400F28ED08EF28C7EEC13F094EC0BF02A0E7B
:1035D4000601A16F9DEC07F094EC0BF0000E0201C4
:1035E400C21902E1000EC11901E1F8D794EC0BF005
:1035F400230E0601A16F9DEC07F094EC0BF0F29EF4
:103604000D0E376E000E386EC2EC12F00B0E060172
:103614008A6F3F0E8B6F000E8C6F96EC0EF0E5EC0C
:1036240012F0020E06016C6F000E6D6F010E6E6FCC
:10363400000E6F6F490E706F3E0E716F000E726F49
:10364400F8EC12F07A0E0B6EC10E0C6E810E0D6E3C
:103654000D2EFED70C2EFCD70B2EFAD7000000003F
:10366400D80E06018A6F3D0E8B6F000E8C6F96ECA0
:103674000EF0C2EC12F06EEC15F0020E06018A6F29
:10368400000E8B6FF4EC0BF0010E06016C6F000E54
:103694006D6F010E6E6F000E6F6F8D0E706F3E0EAC
:1036A400716F000E726FF8EC12F05C0E0B6E510E1F
:1036B4000C6E600E0D6E0D2EFED70C2EFCD70B2E4D
:1036C400FAD700009D8AA38AF28CF28ED08E05016F
:1036D400676B686B0D0E376E000E386EC2EC12F01D
:1036E4006EEC15F00D0E376E000E386E690E356EE9
:1036F400000E366E7EEC13F06E0E0601216F050E81
:10370400226F21C68AF622C68BF6BE0E8C6F3D0E42
:103714008D6F000E8E6FB4EC0EF0040E06012125A1
:10372400E16E000E2221E26E006A83BE002A300E92
:10373400002600C0E6FF0D0E2125E16E000E2221B9
:10374400E26E006A87B6002A300E002600C0E6FF4B
:10375400010E6C6FD7DC00C055F501C056F500C0F2
:103764006CF601C06DF6F00E06016E6F050E6F6FFC
:1037740097EC16F021C68AF622C68BF6F00E8C6FF3
:10378400050E8D6FBBEC09F021C68AF622C68BF6B6
:103794007AEC0BF094EC0BF0E2EC16F06E0E0601F2
:1037A400216F050E226F21C68AF622C68BF65E0EA5
:1037B4008C6F3F0E8D6F000E8E6FB4EC0EF0030E07
:1037C40006012125E16E000E2221E26E006A83BE0D
:1037D400002A300E002600C0E6FF080E2125E16E07
:1037E400000E2221E26E006A87B6002A300E0026FF
:1037F40000C0E6FF55C56CF656C56DF6F00E6E6F4B
:10380400050E6F6F97EC16F021C68AF622C68BF66A
:10381400F00E8C6F050E8D6FBBEC09F0010E8A6FF4
:10382400000E8B6F010E8C6F000E8D6F21C68EF60D
:1038340022C68FF6EFEC0AF0020E06016C6F000E42
:103844006D6F010E6E6F000E6F6F9E0E706F3E0EE9
:10385400716F000E726FF8EC12F0020E06018A6F9F
:10386400000E8B6F080E8C6F000E8D6F1D0E8E6F09
:10387400000E8F6FEFEC0AF01F0E0B6E710E0C6EC4
:103884001E0E0D6E0D2EFED70C2EFCD70B2EFAD766
:103894000000000E0201C21902E1000EC11908E184
:1038A400000E0301525D02E1020E515D01E2F1D707
:1038B4000301000E521902E1020E51196BE1F00EE0
:1038C40006018A6F050E8B6F970E8C6F3F0E8D6FFE
:1038D400000E8E6FB4EC0EF03D0E06016C6F000E00
:1038E4006D6FF00E6E6F050E6F6F070E706FF0EC5C
:1038F4000FF0000E011802E1000E001803E1E4ECE1
:103904000EF009D02E0E06018A6F3D0E8B6F000E4D
:103914008C6F96EC0EF0F00E06018A6F050E8B6F1D
:103924009F0E8C6F3F0E8D6F000E8E6FB4EC0EF0F9
:10393400C30E06016C6F020E6D6FF00E6E6F050EF6
:103944006F6F070E706FF0EC0FF0000E011802E1BC
:10395400000E001800E1200E0601A16F9DEC07F097
:1039640015EC11F000C031F001C032F0000E011866
:1039740002E10A0E001805E189EC13F0F1EC16F0EF
:1039840009D00E0E06018A6F3D0E8B6F000E8C6FF0
:1039940096EC0EF0000E05016A1902E1010E691998
:1039A4006EE16EEC15F0FD0E06018A6F3E0E8B6F14
:1039B400000E8C6F96EC0EF0C10E06018A6F000E9D
:1039C4008B6F7AEC0BF094EC0BF0E2EC16F0F00E4B
:1039D40006016C6F050E6D6FC10E6E6F000E6F6F7A
:1039E400100E706F000E716F21EC10F0010E6C6FF1
:1039F400000E6D6F010E6E6F000E6F6FEF0E706F25
:103A04003E0E716F000E726FF8EC12F0020E06019A
:103A14008A6F000E8B6F010E8C6F000E8D6FF00E8F
:103A24008E6F050E8F6FEFEC0AF03D0E0B6EE10EFC
:103A34000C6E3F0E0D6E0D2EFED70C2EFCD70B2EEA
:103A4400FAD700000000C10E06016C6F000E6D6F06
:103A54002A0E6E6F000E6F6F040E706FF0EC0FF095
:103A6400000E011802E1000E001807E1C50E060160
:103A74006C6F000E6D6F65EC10F0C2EC12F06EEC22
:063A840015F034D6FFD757
:103FAE0010EE1DF01C0E006E010E016E6B0EF66E05
:0E3FBE003D0EF76E000EF86EC3EC10F0120010
:103A8A002055415254312033383430302C382C4EA2
:103A9A002C3120436C69636B657232204D696B72FD
:103AAA006F6275732332205243362C524337203CBF
:103ABA002D20504C32333033202D203E7465726DE8
:0E3ACA00696E616C205642524159200D0A006F
:103AD80020536F75726365204D696B726F43204385
:103AE8006C69636B6572325F31384638374A3530F6
:103AF8005F4750535F434F4D5041535F55424C4FC2
:103B0800585F374E5F4C43445F4849445F5F3136E6
:093B1800303930332E630D0A0030
:103B210050726F6A6574203A20436C69636B6572E9
:103B3100325F31384638374A35305F4750535F433B
:103B41004F4D5041535F55424C4F585F374E5F4C7C
:103B51004344323131395F313630392E6D63707003
:043B6100690D0A00E0
:103B65002055415254322031393230302C382C4EC8
:103B75002C3120436C69636B657232204D696B7221
:103B85006F4275732331205247312C524732203C06
:103B95002D3E204750532055424C4F5820374E0D4F
:023BA5000A0014
:103BA7002048617264776172653A200D0A20436C80
:103BB70069636B6572322031384638374A353020B1
:103BC7005375727669766F72202B204750532D43B9
:103BD7004F4D5053202055426F7820374E0D0A0025
:103BE700204469726563746F7279203A20433A5FA3
:103BF7004D696B726F435F4D657350726F6A657481
:103C0700735F4D696B726F435F31384638374A359A
:083C1700305F4750530D0A0015
:103C1F000D0A546573742064757265652054696D5F
:103C2F0065723320696E697469616C6973E920E0AC
:103C3F00203130307834306D53202C736F697420FD
:073C4F00347365630D0A00E8
:103C56005541525431203139323030203C2D2D2DF2
:103C66002070726F6C696669782D3E205465726D9E
:0B3C7600696E616C205043200D0A00B5
:103C810020464F53433D384D687A20696E74657202
:103C91006E65207820504C4C203D3E2034384D68D4
:063CA1007A20200D0A004C
:103CA70020436865636B2070726573656E6365207A
:103CB7004C43443231313920617420402030783709
:043CC700340D0A00AE
:103CCB00554152543220313932303020203C2D2D89
:103CDB003E204750532055424C4F5820374E0D0A2B
:023CEB002000B7
:103CED00204C696169736F6E204D6F64756C652032
:103CFD004750532055424C4F5820374E3A200D0A0D
:013D0D0000B5
:103D0E0042414420526563657074696F6E206F7511
:103D1E00204465636F64616765204747410D0A0063
:103D2E0042414420526563657074696F6E206F75F1
:103D3E00204465636F64616765204747410D0A0043
:103D4E0020496E697420493243322048617264778B
:0D3D5E00617265203430304B687A0D0A0028
:093D6B0030312F30312F313600C8
:043D7400000000004B
:053D78004364653D00FD
:023D7D00200024
:023D7F00000042
:023D8100200020
:023D83006400DA
:023D85000D002F
:103D8700204465636F6465205472616D65204E4DF4
:0C3D97004541204750474741200D0A00DD
:103DA300464F53433D34384D485A2020504C4C2005
:0B3DB30061637469766520200D0A0032
:103DBE004250313D202020203B4250323D202020D9
:0A3DCE0020203B204541313D20003C
:103DD8002041726D652049542055415254312026A6
:093DE8002055415254320D0A002D
:103DF100504F525420555342204849442054657233
:093E01006D696E616C200D0A0070
:103E0A00204C696169736F6E20504943203C2D3EF6
:083E1A002050433A200D0A007C
:103E220020496E6974204C434420323131392032AA
:063E32007831360D0A0094
:103E3800203130302078203430203D2034736563C1
:013E48000079
:103E4900496E69742041444320737572204541319C
:013E59000068
:103E5A005554433A2020204820204D20205320202A
:013E6A000057
:103E6B004C4F4E3A202020202020202020202020A4
:013E7B000046
:103E7C004C41543A2020202020202020202020209B
:013E8C000035
:103E8D0041726D6520496E74657272757074732020
:013E9D000024
:103E9E0044617465203A20202020202020202020FC
:013EAE000013
:103EAF00416C74697475643A2020202020202020F2
:013EBF000002
:103EC000496E69742054696D6572332034306D53C6
:013ED00000F1
:103ED100436865636B204465766963652040200013
:0E3EE100206973206E6F7420666F756E64002A
:0E3EEF0055415254312052656375203A20002F
:0E3EFD0055415254312052656375203A200021
:0D3F0B0020496E697420414443310D0A00C5
:0C3F1800204461746520524D433D2000A0
:0C3F24002020202048444F50203A20006C
:0C3F300020202020204C6174203A20004A
:0C3F3C002020202020416C74203A20003E
:0B3F4800202020536174656C3A2000BB
:0B3F5300202020204C6F6E203A200040
:0B3F5E0042313D2E2042323D2E20005B
:0A3F6900202020204669783A20004D
:0A3F730020666F756E64204F4B004E
:093F7D0032202048415244570053
:093F86004A4A2F4D4D2F41410024
:083F8F00206F6E20493243004F
:083F9700244750524D432C0059
:083F9F002447504747412C0064
:073FA700205574633A20006D
:020000040001F9
:06FFF800AEF7C4FFF8FFA4
:00000001FF
